:020000040000FA
:100000008316031300308600F830870041202E202D
:100010001E2015200C20072803178312103091078B
:1000200021208312031386000800212012081002E9
:10003000031D1B281D28910A152808000030910077
:1000400008008312031711088D0083168C130C14FB
:100050000C18282883120C0892000800831203133E
:10006000871D30288719322807080317831290004C
:100070000310900C0310900C0310900C0310900CC4
:100080000800831203170530910021200530120269
:10009000031D51281E3091002120673012020319E0
:1000A000F42800308D0000308C00F92001308D00E4
:1000B00001308C00F92002308D0002308C00F920D4
:1000C00003308D0003308C00F92004308D000430A3
:1000D0008C00F92005308D0005308C00F9200630A9
:1000E0008D0006308C00F92007308D0007308C0021
:1000F000F92008308D0008308C00F92009308D007F
:1001000009308C00F9200A308D000A308C00F9206B
:100110000B308D000B308C00F9200C308D000C3032
:100120008C00F9200D308D000D308C00F9200E3040
:100130008D000E308C00F9200F308D000F308C00B8
:10014000F92010308D00FC308C00F92011308D002A
:1001500060308C00F92012308D00DA308C00F920EC
:1001600013308D00F2308C00F92014308D00663091
:100170008C00F92015308D00B6308C00F920163037
:100180008D00BE308C00F92017308D00E0308C00DF
:10019000F92018308D00FE308C00F92019308D00C8
:1001A000F6308C00F9201A308D00FD308C00F920DB
:1001B0001B308D0061308C00F9201C308D00DB304D
:1001C0008C00F9201D308D00F3308C00F9201E309A
:1001D0008D0067308C00F9201F308D00B7308C0007
:1001E000F920831603170C118312031302308600C3
:1001F0000800831603170C1555308D00AA308D00AA
:0E0200008C148C1801290C12831203170800AD
:02400E00F13F80
:00000001FF
